:020000040800F2
:10500000381C0020D5500008B5900008978600088D
:105010000000000000000000000000000000000090
:10502000000000000000000000000000D19D00080A
:105030000000000000000000899B00080D9F000890
:10504000E7500008E7500008E7500008E750000864
:10505000E7500008255C0008E7500008E75000080A
:1050600000000000E7500008315B0008E75000082E
:10507000E7500008C58B000800000000E75000085A
:1050800000000000E75000080000000000000000E1
:10509000E750000800000000E7500008E750000853
:1050A000E7500008E7500008E7500008A1A90008F1
:1050B000E7500008E7500008000000000000000072
:1050C0000348854600F07EFC00480047A1BA00086E
:1050D000381C00200448804704480047FEE7FEE7EC
:1050E000FEE7FEE7FEE7FEE7CD9F0008C15000089F
:1050F00030B50B46014600202022012409E00D4670
:10510000D5409D4205D31D469540491B25469540F7
:1051100040191546521E002DF1DC30BD70B500243B
:105120002546002801DA01244042002901DA012540
:105130004942FFF7DDFFAC4200D04042002C00D0D6
:10514000494270BDF0B51FB40646002082B0054646
:105150004024019100901BE0019922460F46304601
:1051600000F06CFB049A059B801A994110D31046FD
:105170001946224600F052FB361A8F41019722460B
:1051800001200021009F00F049FB38184D4100909C
:105190002046641E0028DFDC019B00982946324629
:1051A00007B0F0BD03460B439B0703D009E008C9D5
:1051B000121F08C0042AFAD203E00B780370401CC7
:1051C000491C521EF9D27047D2B201E00270401C55
:1051D000491EFBD270470022F6E710B513460A4677
:1051E00004461946FFF7F0FF204610BD30B50446CF
:1051F0000020034600E05B1C934203D2E05CCD5CE0
:10520000401BF8D030BDF8B502464A40D40F4200EA
:105210004B0052085B089A4202D2024608461146E9
:105220004A0023D0C30D4A00DDB2120EAD1A202D64
:1052300035DA49020126490AF6058A19002C00D000
:10524000524220214F1B1146B9402A411018C20D6D
:105250009A4221D0002C17D0012D08DCDA05801AE3
:10526000D20F8019D207DBB200F014FBF8BDDA05CB
:10527000801A012340001B06C01880185A4280186B
:10528000CA0F1043490007E04908C2071143DA0575
:10529000801A80194008801800F0F4FAF8BD610007
:1052A0000122511A001BF7E70122D2075140AAE759
:1052B0000122D2075040A6E770B502464A40D50FFA
:1052C00040004A00ED0740085208002814D0002A88
:1052D00012D0C40DD30D41020120C0055202490A6B
:1052E000520AE41A091812187D34914201D3641C41
:1052F00000E04900002C01DA002070BD002391423B
:1053000001D3891A0343400849000028F7D1002936
:105310000AD0914202D10121C90705E0914201D290
:10532000012101E00121C943E005C018401900F046
:10533000A9FA70BDF0B507460846584087B0C00FBF
:10534000049048000E46590040084908BC1A88419C
:1053500005D2384631461E4617460B4602465800CF
:10536000400810434CD0300D039040055900400DCB
:10537000490D0590401A0290402872DA1803012165
:10538000000B09050843019004980092002805D0FD
:1053900001995242002088410092019002984021D8
:1053A0000A1A0199009800F039FA05460C466B4636
:1053B00007CB00F054FAC0197141039A0E0D002377
:1053C000D71756401A467A40164344D0049A002A0A
:1053D0002DD0029A012A039A15DC1205C01A9141B8
:1053E00001263605001C7141D20F059ED20700939D
:1053F000019202962A46234600F092FA07B0F0BDC9
:1054000038463146FAE71605224A0F46B218C01A46
:10541000B74101210905001C4F4100187F41114689
:1054200018187941E20F10436D19644113E0E20747
:105430006D0815436408C2071443039A0126120538
:10544000C01A91413605001C7141CE074008304317
:105450004908C01851412A46234600F054FACDE7C6
:10546000FFE7049801224000C117121A00238B4164
:1054700004983146C417381AA141EEE730B401242C
:10548000E407634030BC55E730B40124E4076140D1
:1054900030BC4FE70000E0FFF0B51FB488B00B99B7
:1054A0000998002448400999C00F4900490809910A
:1054B000C0070B990090490049080B910999089879
:1054C000A64608431CD00B990A98084318D009989F
:1054D00001244000420D4800410D099824050003B5
:1054E000000B204309900B980003000B20430B9006
:1054F00050181C494018002201901446104605E03F
:10550000002001460DB0F0BD032801DA034600E09B
:1055100003239C46C11A0AAE0AE05F0008ADED5BAA
:105520004F00F75B7D430027AA187C41491C5B1E96
:105530006145F2DD410004AB5A522104120C0A43CA
:10554000240C401C0828DFDB01980290009970466B
:1055500001910090059B049A0799069800F0E0F9E4
:10556000D0E700000DFCFFFFF0B50C465C4085B0B5
:10557000E40FE40703944C000026640859009446A5
:10558000490802460296224321D062460A431ED0B1
:105590006200570D4A000E032303550D01240246F5
:1055A0002C492405781B1B0B360B4018234326433C
:1055B000614600901C46501AB44103D30098401C29
:1055C000009002E0921800985B41002803DA002066
:1055D000014605B0F0BD00200121090507468646B9
:1055E00011E064461D46141BB54106D36546521BA7
:1055F000B341744607430C43A646CD07400849080B
:10560000284392185B4105460D43EAD110461843E2
:1056100013D06046194650407140084306D060469A
:10562000101AB34106D20122002306E00022012312
:10563000DB0702E00122D2435310009874460105B3
:10564000381C6141029C039D0019694100F05BF91F
:10565000BFE70000FD030000C217C10F504010B5A6
:105660004018CA079623002100F014F910BD10B5A8
:1056700000229623114600F00DF910BD0EB5C21799
:10568000C10F5040CA0740180021054B02930192F8
:1056900000910A460B4600F043F903B000BD00003C
:1056A000330400000EB505490291002100910A461D
:1056B0000B46019100F034F903B000BD3304000043
:1056C000410040020122400AD205090E80187F29BC
:1056D00001DA00207047962903DC9622511AC8404F
:1056E000704796398840704770B5CD0F4A0009035E
:1056F0000123090B1B0519430B4BED070024520D29
:105700009A4201DA002070BD074B34339A4203DC21
:105710009A1A00F093F802E00449511888402C438B
:10572000F1D0404270BD0000FF030000CDFBFFFF41
:105730004A0009030123090B1B051943094B10B546
:10574000520D9A4201DA002010BD064B34339A42C2
:1057500003DC9A1A00F072F810BD03495118884012
:1057600010BD0000FF030000CDFBFFFFC20FD207FA
:10577000400040080BD0C10D0723DB01C9184002CF
:105780000905400A1143C208400711437047002031
:105790000146704710B5002904DB0124E4074042AC
:1057A0008C412146002B04DB1C460123DB075242BF
:1057B000A341994200D1904210BD0000CB0FDB07FE
:1057C000490010B5490802460A4307D00A0D0724CC
:1057D0000903E401090B121B002A01DC002010BDA3
:1057E000C900440F0C43C100E018D205801800F036
:1057F00049F810BD0122D207002800DB101A002949
:1058000000DB511A814270470122D207002800DBD9
:10581000101A002900DB511A8842704710B5202A5F
:1058200004DB0146203A9140002010BD9140202326
:105830009C1A0346E3401943904010BD10B5202A3E
:1058400004DB0846203AD040002110BD0B46D3406F
:10585000D0402024A21A91400843194610BD10B52B
:10586000202A06DBCB170846203A1041C1170B430C
:1058700006E00B461341D0402024A21A9140084371
:10588000194610BD002904DA401C490001D1400826
:105890004000704770B40024050C05D110240004AA
:1058A00002D1002921D01124050E01D100020834B3
:1058B000050F01D10001241D850F01D18000A41C1A
:1058C000002801DB4000641C002908D020252E1B85
:1058D0000D46F540A14000D00121294308430106AF
:1058E0001B1B000ADB1D02D5002070BC7047DB05C6
:1058F000181880180029F8DA401C4900F5D170BC4E
:1059000040084000704710B5002B08DA0024401C06
:10591000614192185B411A4301D14008400010BD1B
:10592000F0B51FB482B005460C0003D0084605F060
:1059300065F902E005F062F9203002460090214648
:105940002846FFF76BFF049B059A04460F46184351
:105950001143084314D0184610431BD0009840212F
:105960000A1A18460599FFF769FF05460E46009A80
:1059700005990498FFF752FF084305D0012004E081
:105980002046394607B0F0BD0020C11705430E433D
:105990002C43374300990E986305401A7905E40AB1
:1059A00000220C43FD0A0A3002D500200146E9E737
:1059B0000105101969410C9C0D9D00196941FFF703
:1059C000A2FFDFE7064C0125064E05E0E36807CCA1
:1059D0002B430C3C98471034B442F7D3FFF774FBC9
:1059E00064BE000884BE000870B58C180578401CA1
:1059F0006B075B0F01D10378401C2A1106D1027896
:105A0000401C03E006780E70401C491C5B1EF9D157
:105A10002B0705D40023521E0DD40B70491CFAE746
:105A20000378401CCB1A921C03E01D780D70491CB2
:105A30005B1C521EF9D5A142D8D3002070BD0000D6
:105A400038B50446074908480068FFF751FB604332
:105A5000009002E00098401E009000980028F9D1C4
:105A600038BD000040420F008401002070B504469C
:105A70000025206880688007800F012807D12068F2
:105A80000068C007C00F002801D0012000E00020FE
:105A9000002839D1206880681C490840002801D1BD
:105AA000012000E00020002809D1606D102108438A
:105AB0006065A06D01210843A065012070BD2068CC
:105AC000806801210843216888600120FFF7B8FF42
:105AD00001F014FA05460EE001F010FA401B0A2806
:105AE00009D9606D102108436065A06D012108434C
:105AF000A0650120E2E720680068C007C00F01210F
:105B0000484048400028E7D00020D7E71700008031
:105B100010B502460B460020002103E0545C241817
:105B2000A0B2491C9942F9D3C443A0B210BD0000F1
:105B300010B5034800F0E0FE024800F0DDFE10BDA5
:105B4000D81700209017002030B51C25446C2C403D
:105B50000125A540046C6560046863608468102CAE
:105B600004D10468A2600468E16003E00468A160F5
:105B70000468E26030BD000001201749487202202D
:105B80001649487203201649487204201549487284
:105B9000114815490A7842714978817110481249B3
:105BA0000A784271497881710C480F490A7842702D
:105BB000497881700B480C490A78427049788170A5
:105BC0000A4809490A7842704978817006490A787A
:105BD0004271497881717047B81100201612002077
:105BE000DA110020CC110020400100202C120020EE
:105BF00010B504F0C1F8202004F076F9012005F07A
:105C000019FC002004F070F9044805F081FA0448FA
:105C100005F0B2FD002005F0EFFD10BD6100002091
:105C20008380000010B501210520000701F056F91E
:105C3000002802D000200C49086002210B4801F026
:105C40004DF9002809D108490860094800880A214F
:105C500048430849088004F0B5FE012001F038F8F7
:105C6000022001F035F810BD7C0100200004005036
:105C70005C010020700100207047000000210A4AEA
:105C800051610A494968012252021143074A516091
:105C90001146496808221143044A51600021C20993
:105CA000D20111607047000020180020002002403F
:105CB0007FB504460D460020039000F0C1FF002090
:105CC00000900194E809029003A9684600F03AFFA9
:105CD000002804D000F07CFF002004B070BD00F06C
:105CE00077FF0120F9E710B50346002002E01C5CB5
:105CF0000C54401C9042FAD310BD000000203949DA
:105D00008969FF2201321140914208D1364949691F
:105D100002221143344A5161FF21013108433149C4
:105D20008969012252021140914208D12E494969E4
:105D3000012211432C4A516101214902084329499A
:105D40008969012292021140914208D1264949698C
:105D500008221143244A5161012189020843214943
:105D600089690122D2021140914208D11E49496934
:105D7000042211431C4A51610121C90208431949F7
:105D80008969012252031140914208D1164949699B
:105D900010221143144A516101214903084311495A
:105DA0008969012252041140914207D10E49496983
:105DB000202211430C4A5161202108430949896975
:105DC000012212041140914208D107494969402239
:105DD0001143054A516101210904084301498861C1
:105DE00070470000002002402018002070B50446D3
:105DF00001F084F805460BE0601C002808D0002C58
:105E000004D001F07BF8401BA04201D9032070BDF3
:105E10001F488069C007C00F0028EDD11C48806969
:105E200002210840022801D1194988611848806977
:105E3000FF2101310840884223D01548806949007C
:105E4000084088421DD012488069490008408842B5
:105E500017D00F48806949000840884211D00C488B
:105E600080698900084088420BD00948806909018F
:105E70000840884205D00648806949100840884299
:105E800003D1FFF73BFF0120C1E70020BFE700007F
:105E900000200240F0B585B006460F4614460025A6
:105EA000029601970020009000F0CAFE13E00198CE
:105EB000006803900220039A029900F099FE009076
:105EC0000098002800D008E00298001D0290019878
:105ED000001D01902D1DA542E9D300BF00F078FE02
:105EE000A54202D2002005B0F0BD0120FBE7000072
:105EF0000246002108E04800064B185A904201D1A2
:105F000008467047481CC1B2034800788142F2DB62
:105F100000BFF6E72614002028010020FEB50C483B
:105F200001F0FAF980B202900298FFF7BBFB044639
:105F3000084A094BFFF7B0FA0022084B0191009084
:105F4000FFF712FB0646FFF7F3FB80B2FEBD000031
:105F500088160020F853E3A59B843E4000408F4004
:105F600010B54B480078002803D00020484908703D
:105F700002E0012046490870464845490A784270C7
:105F80004978817044490A784271497881710520C5
:105F900040494872962005F0DDFB4B20C00005F01B
:105FA000F5FB00223B490C2005F0F2FC00210C20FF
:105FB00005F002FD022005F027FC00BF00210F20A4
:105FC00005F020FB35490860354908400028F5D028
:105FD00032480068401C002801D103F0A9F82F487E
:105FE000006801218903084000283FD08122D201A6
:105FF00000210F2005F085FC0021102005F002FB98
:106000004406640E21460022264805F04BFB254835
:10601000407A05283AD102221F492248401DFFF745
:10602000E5F8002832D11F48807A1F490870042201
:106030001C49491C1D48FFF7B5F81C48006800F0D2
:1060400043F81B49088018480078420015490B3175
:106050001848FFF7A7F816480088174909884843E9
:10606000164908800220164908700FE01049088878
:106070000988491E0E4B198012490988FFF74EF80E
:106080000D480088414388B20C49088010BD0000CB
:10609000380100202C120020400100207000002058
:1060A00000D027247C12002028010020300100208D
:1060B000FC00002026140020520100204E01002088
:1060C000600000205401002070B50646174801F01A
:1060D00023F9C5B22846E917C90E09184911490123
:1060E000691ACCB209E03046E040C007C00F002872
:1060F00001D1204670BD601CC4B20D4800888442A6
:10610000F1DB012409E03046E040C007C00F002861
:1061100001D12046EEE7601CC4B2054800888442E5
:10612000F1DB03480078401EC0B2E3E78816002088
:106130005401002010B50B4800F074FB0A210948F7
:1061400000F0FAFA074800F0A1F9012149020840DD
:10615000884204D1034800F09CF980B210BD00BF12
:10616000FCE700002C160020F0B587B000220121CA
:10617000424800F0BCFEFFF7DDFF0546FFF777FA67
:1061800004463F49FFF798F83E490860012211464E
:106190003A4800F0ACFE3B480068FFF7E7FA0446D7
:1061A0000022394BFFF7F6FA5ED83848007800280D
:1061B00021D0002035490870FFF7BCFF0546FFF7E6
:1061C00056FA04462E49FFF777F82E49086008462C
:1061D0000068FFF7CBFA044600222B4BFFF74EF97D
:1061E00000222B4B05910490FFF756F90646FFF766
:1061F000E5FA2849086023480068FFF7B7FA064621
:106200000022214BFFF73AF90446234A234BFFF7BC
:1062100043F9039102901F480068FFF7A7FA04466C
:106220001D4A52421E4BFFF737F901910090039B24
:10623000029AFFF77FF805910490FFF7BFFA15491E
:106240000860184913480068FFF7DEFA02D21548C3
:106250001049086000210F480068FFF7CBFA06D20A
:1062600000200C49086002E000200A490860094843
:106270000068FFF725FAC0B207B0F0BD0004005077
:1062800000401B442800002000000C40300000208B
:1062900000E064402C0000203333333333B330400C
:1062A000CCCCEC3F0000C842F8B5044600250026DF
:1062B000002700BF5020005D012801D10220F8BD59
:1062C00001215020015500BF206880688007800FA1
:1062D000012806D1206800680840002801D001206C
:1062E00000E00020002841D1606DFF21013188438A
:1062F0000221084360652068C0688707BF0F2068D7
:10630000C068800880002168C8602068806801211A
:10631000C90708432168886000F0F0FD064611E0D7
:1063200000F0ECFD801B0A280CD9606D0221884327
:1063300010210843606500BF00215020015500BFB7
:106340000120BCE720688068C00FC0070121C90791
:106350008842E5D02068C06838432168C860606D15
:106360000221884301210843606504E0606D20211B
:1063700008436065012500BF00215020015500BF82
:1063800028469CE770B504460D4600BF5020005DCE
:10639000012801D1022070BD01215020015500BF0C
:1063A0002068806804210840800800280AD0606DB9
:1063B00020210843606500BF00215020015500BF27
:1063C0000120E8E72D496868884229D02068806A62
:1063D00029684903490B08432168886228684003FB
:1063E000400B2749084001218904884208D12548EB
:1063F000806849010843234988600A20FFF720FB91
:1064000028684003400B2049084001214904884284
:106410002CD11C488068490108431A49886025E04E
:106420002068806A29684903490B8843216888628B
:1064300028684003400B1249084001218904884222
:1064400005D110488068490188430E498860286852
:106450004003400B0C49084001214904884205D102
:1064600008488068490188430649886000BF0021C8
:106470005020015500BF00208DE7000001100000F2
:106480000000044800270140000002440146486D16
:10649000704701460868006C7047000010B504465C
:1064A000002C01D1012010BD606D002806D1A0652F
:1064B000002150200155204600F00EF9606D10219A
:1064C0000840102806D02068806804210840800811
:1064D00000280AD0606D10210843606500BF0021CC
:1064E0005020015500BF0120DDE7606DFF21013123
:1064F0008843022108436065206880688007800F18
:10650000012807D120680068C007C00F002801D00B
:10651000012000E0002000283AD100BF03218907B4
:106520006068884207D049426068884203D04900C9
:10653000606888420CD1206800698000800821686A
:10654000086120680069616808432168086112E0F9
:106550002068006980008008216808615C488068C4
:106560000F21890488435A49886008468068616819
:1065700008435749886000BF2068C06818218843D5
:106580002168C8602068C068A16808432168C860A5
:106590004F4880680121490688434D498860084674
:1065A0008068A18E49060843494988602068806850
:1065B000012109070840002804D1206880680843A9
:1065C000216888602068C068424908402168C86026
:1065D0002169E068022901D1042100E0002108437B
:1065E0002021095D490308432C21095D4900084326
:1065F000216B0843A16989030843E169C903084382
:106600002168C96808432168C860FF21C231606AF7
:10661000884207D0A16A606A08432168C9680843B4
:106620002168C8602120005D012813D12020005D71
:10663000002807D12068C0680121090408432168A7
:10664000C86007E0606D202108436065A06D0121EE
:106650000843A065E06B012817D120680069FF217D
:106660008900884321680861216C606C0843A16C33
:1066700008432168096908432168086120680069A6
:1066800001210843216808610BE020680069C00708
:10669000C00F002805D0206800694008400021682C
:1066A000086120684069C008C0002168486120680E
:1066B0004069A16B0843216848610020A065606DB6
:1066C000022188430121084360650020EBE60000B9
:1066D000002701401902FEFF10B586B004461421C0
:1066E00001A8FEF778FD1249206888421ED11148A2
:1066F000406B491508430F49486300BF0846C06A0C
:10670000012108430B49C8620846C06AC007C00F90
:10671000009000BF00BF02200190032002900020E3
:10672000039001A90520000700F0E2FA06B010BDB1
:106730000024014000100240F8B504460D46002632
:1067400000276069082801D1082711E02068C06887
:10675000C007C00F00280AD0606D20210843606583
:1067600000BF00215020015500BF0120F8BD0C27BB
:1067700000F0C4FB064614E0681C002811D0002D70
:1067800004D000F0BBFB801BA8420AD9606D042135
:106790000843606500BF00215020015500BF032061
:1067A000E4E72068006838400028E5D0606D0121EA
:1067B0004902084360652068C068032189020840D7
:1067C000002826D12020005D002822D12068006802
:1067D0000821084008281CD120688068042108404E
:1067E000800800280DD1206840680C21884321686A
:1067F0004860606DFF2101318843012108436065D5
:1068000007E0606D202108436065A06D0121084309
:10681000A065A069002802D10C2021680860002032
:10682000A4E7000070B504460025206880680421B4
:106830000840800800282BD100BF5020005D0128AF
:1068400001D1022070BD01215020015500BFE06937
:10685000012803D02046FFF709F90546002D18D17D
:10686000606D0D490840FF2101310843606500203B
:10687000A06500BF00215020015500BF1C202168E9
:10688000086020688068042108432168886000E06F
:1068900002252846D6E70000FEF1FFFF70B504464A
:1068A00000252520005D022803D00420E063012597
:1068B00020E0206800680E21884321680860206875
:1068C000006840084000216808601C21606C084096
:1068D00001218140206C416001212520015500BF2C
:1068E00000212420015500BFA06B002802D02046C3
:1068F000A16B8847284670BD70B50446206C0568BA
:10690000206806681C20616C0140042088402840F3
:1069100000281DD004203040002819D020680068CD
:1069200020210840002805D1206800680421884300
:10693000216808601C21606C084004218140206CA3
:106940004160206B00285AD02046216B884756E0D2
:106950001C20616C0140022088402840002825D07E
:1069600002203040002821D0206800682021084003
:10697000002808D1206800680A218843216808603F
:106980000121252001551C21606C08400221814015
:10699000206C416000BF00212420015500BFE06A47
:1069A00000282CD02046E16A884728E01C20616C32
:1069B0000140082088402840002820D0082030408E
:1069C00000281CD0206800680E21884321680860D8
:1069D0001C21606C084001218140206C4160012035
:1069E000E06301212520015500BF0021242001552D
:1069F00000BF606B002802D02046616B884770BDE5
:106A000070B50446002C01D1012070BD244A2168D4
:106A1000881A1421FEF76CFB800060642048083857
:106A20002064022125200155206805681D48054085
:106A3000E168A06808432169084361690843A169C6
:106A40000843E1690843216A08430543206805605B
:106A500001218903A068884217D011487830806AE4
:106A60001C22616C11400F228A4090430C497831FE
:106A700088621C22616C1140606888400849783146
:106A8000896A08430649783188620020E063012161
:106A9000252001550021242001550020B5E70000E4
:106AA000080002400F80FFFFF8B504460D46164669
:106AB0001F460020009000BF2420005D012801D166
:106AC0000220F8BD01212420015500BF2520005DD2
:106AD00001282DD10221252001550020E0632068E6
:106AE000006840084000216808603B46324629465D
:106AF0002046FFF729F8206B002806D020680068A0
:106B00000E210843216808600BE02068006804211A
:106B1000884321680860206800680A2108432168CA
:106B2000086020680068012108432168086006E0C9
:106B300000BF00212420015500BF022000900098D2
:106B4000BFE70000F8B504460E460127002500BF48
:106B50001C48007C012801D10220F8BD0120194900
:106B6000087400BF1848FFF741F90746002F22D1EB
:106B7000401E3060656817E02846FFF77FF812482E
:106B8000FFF734F9074611484068082188430F4948
:106B9000486008464068491588430C494860002F02
:106BA00001D0356006E08035A068C00161684018FA
:106BB000A842E1D800BF00BF00200249087400BF0E
:106BC0003846CAE72018002050C3000000200240C9
:106BD0000648406802210843044948600846406866
:106BE000012108430149486000207047002002400D
:106BF000F8B507460C461546012600BF0E48007C36
:106C0000012801D10220F8BD01200B49087400BF02
:106C10000A48FFF7EBF80646002E06D10649486100
:106C200025600648FFF7E2F8064600BF002002494B
:106C3000087400BF3046E6E72018002050C300006B
:106C40001D484068C007C00F002816D000BFEFF3F2
:106C50001080014600BF72B61848174AD060184825
:106C6000D06000BF81F3108800BF10464068C007A5
:106C7000C00F002801D0012070470F484068022251
:106C80001040022815D100BFEFF31080014672B604
:106C90000C48094A10610C481061084680F31088BE
:106CA00000BF1046406802221040022801D1012096
:106CB000E2E70020E0E7000000200240EFCDAB89D2
:106CC00005040302BFAE9D8C161514137047000017
:106CD00010B50446054840692040002804D0034808
:106CE00044612046FFF7F2FF10BD000000040140A0
:106CF00070B50346002200240020DAE00126964009
:106D00000D6835402C46002C77D04D68022D02D0FE
:106D10004D68122D15D1D508AE001D462035A85955
:106D20005507EE0E0F25B5400646AE4330465607D2
:106D3000F60E0D69B5402843D508AD001E46203635
:106D400070514D68012D08D04D68022D05D04D6859
:106D5000112D02D04D68122D18D1986856000325C8
:106D6000B5400646AE4330465600CD68B540284390
:106D700098605868012595400646AE433046102677
:106D80004D6835402D0995402843586018685600D5
:106D90000325B5400646AE4330460D79AD07AD0F2D
:106DA0005600B54028431860D86856000325B54002
:106DB0000646AE43304656008D68B5402843D8603D
:106DC000012636074D683540B54271D13C4D6D6B9B
:106DD000012635433A4E75633A4D9608B600A859D8
:106DE00095072E0F0F25B5400646AE4330460525C4
:106DF0002D07AB4202D1002515E059E0324DAB42E0
:106E000001D101250FE0314DAB4201D102250AE04D
:106E10002F4DAB4201D1032505E02E4DAB4201D1F0
:106E2000052500E006259607360FB5402843254D79
:106E30009608B600A851284D28680546A54328465F
:106E4000012636044D683540B54202D1054625433A
:106E50002846214D286068680546A5432846012636
:106E600076044D683540B54202D105462543284693
:106E7000194D6860A8680546A543284601263605D1
:106E80004D683540B54202D1054625432846124D8E
:106E9000A860E8680546A5432846012676054D68A2
:106EA0003540B54202D10546254328460A4DE860E3
:106EB000521C0D68D540002D00D01FE770BD0000AA
:106EC000001002400800014000040050000800507B
:106ED000000C0050001C00500004014002461369E1
:106EE0000B40002B01D0012000E000207047002A59
:106EF00001D0816100E081627047000001480068B4
:106F0000704700008001002002480068401C0149D1
:106F1000086070478001002010B500240848006810
:106F20004021084306490860002000F00BF80028C3
:106F300001D0012401E000F025FA204610BD000038
:106F40000020024070B5044600257D21C900094893
:106F50000068FEF7CDF8064601F0D4F8002801D00D
:106F6000012504E000222146501E00F033FA284695
:106F700070BD0000840100207047704770B5054661
:106F80003C480078401C3B49087001203A49087091
:106F90003A480088401C394908803948008802F086
:106FA0005BFF3849C888FEF762FB06463649FEF7A4
:106FB00083F90446354801682046FEF724F9334931
:106FC000086002213248FFF789FF002819D12D49B6
:106FD000C888FEF74CFB06462B49FEF76DF90446C0
:106FE0002C4801682046FEF70EF92A4908602A4914
:106FF00028480068FEF708FC06D828482849C860D9
:1070000002E0002023490860264920480068FEF776
:10701000FBFB03D201202449087002E00020224932
:1070200008701849498F481EFEF716FB044617489A
:1070300001682046FEF7DEFB09D81C4800780028CE
:1070400005D01B48C079012108431949C8710D4971
:10705000488FFEF70CFB04460C4801682046FEF7FB
:10706000C9FB05D211480078002801D004F0A8FD22
:1070700070BD00007A0100204D0100206801002051
:107080004E010020B80D002000007A447C01002051
:1070900000040050740100200000A0400400FA0524
:1070A00000ED00E0000040402E01002062010020C1
:1070B0002C120020704710B50446002C01D101208D
:1070C00010BD02212E200155204601F083FD2046EF
:1070D00000F0F4F800212E20015500BF2D200155AD
:1070E00000BF0020ECE77047704710B504462068E9
:1070F0000068C007C00F01214840484000280CD05C
:1071000020688068084048404840002805D0012099
:10711000216848602046FFF731FF2068006802219F
:107120000840400800280BD02068806808404008CC
:10713000002805D00220216848602046FFF71CFF88
:107140002068006804210840800800280BD02068CF
:10715000806808408008002805D004202168486025
:10716000204600F00DF92068006808210840C0089A
:1071700000280BD0206880680840C008002805D08F
:107180000820216848602046FFF794FF20680068C7
:1071900010210840000900280BD0206880680840B2
:1071A0000009002805D01020216848602046FFF71C
:1071B000E4FE2068006820210840400900280BD028
:1071C0002068806808404009002805D020202168F8
:1071D00048602046FFF788FF20680068402108408B
:1071E000800900280BD020688068084080090028AA
:1071F00005D04020216848602046FFF774FF10BD8D
:1072000070B50446002C01D1012070BD60680128D2
:1072100000D100BF26496069884200D000BF2E20FF
:10722000005D002805D100212D200155204600F0E9
:1072300059F802212E2001552068C5686068012890
:1072400003D08905A06A884203D11E2128468843BD
:10725000054617496069884201D01648054016481E
:107260000540A16860680843216A0843616A0843D1
:10727000A16A084305436068012804D00121C905BB
:10728000A06A884203D1E1682069084305430849A0
:107290006069884205D06169A0690843E1690843D3
:1072A00005432068C56001212E2001550020ACE770
:1072B000FFFF00003F1FFFFFF8F119FF10B5044664
:1072C00006492068884208D10548806B4000400884
:1072D000034988630D2000F065F810BD007C004074
:1072E0000010024010B504460949206888420DD1BB
:1072F0000848806B4905084306498863002201213C
:107300000D2000F067F80D2000F058F810BD0000C7
:10731000007C00400010024001460868C0697047C8
:1073200010B5034602242E20C454144800682407D4
:107330002043124C20601868C0680124E4042043F4
:107340001C68E06018688068012420431C68A06005
:1073500018680069012420431C6820611868816155
:107360001868426118680069042420431C68206181
:1073700001242E20C454002010BD00000004014050
:10738000704700000648406B0121084304494863E8
:107390000846806B09040843014988637047000070
:1073A0000010024000BFC206D20E01219140024AE5
:1073B000116000BF7047000080E100E000BFC2061E
:1073C000D20E01219140024A116000BF70470000B7
:1073D00000E100E070B504460D46164629462046F9
:1073E00001F06AFE70BD0000024949688143014A0C
:1073F000516070470070004003480068FF21013170
:10740000084301490860704700700040024949681C
:107410000143014A5160704700700040074800680E
:107420000221084305490860054800690421084312
:107430000349086100BF00BF30BF704700700040C3
:1074400000ED00E010B5024600200E4B18688008E1
:1074500080000346134318460A4B18600A4B1B6909
:1074600004242343084C2361012901D130BF02E0E9
:1074700040BF20BF20BF044B1B690424A343024C20
:10748000236110BD0070004000ED00E0F8B5044637
:1074900020212068084020287CD12068084020282E
:1074A00000D100BF00278148806B012109070840F7
:1074B000002805D17D48806B08437C4988630127FB
:1074C0007B480068FF2101310840002816D1784828
:1074D0000068084376490860FFF710FD064606E09D
:1074E000FFF70CFD801B642801D90320F8BD70480C
:1074F0000068FF21013108400028F1D06B48056881
:10750000032109050D4060680840A8420DD009110B
:1075100060680840884208D1644800680121490435
:107520000840884201D10120E0E76048403000690E
:107530000321090408400546002D3DD0606808403D
:10754000A84239D0202120680840202834D157484B
:107550004030006903210904884305465348403000
:1075600000690121C90408435049403108610846B7
:1075700000690121C90488434C494031086108462B
:107580000561801528408915884215D1FFF7B6FCA2
:10759000064608E039E0FFF7B1FC801B4549884208
:1075A00001D90320A2E74148403000690121490286
:1075B0000840400A0028EED000BF00BF03210904A4
:1075C0006068084088420AD1384800680901884349
:1075D000032212056168114008433449086000BF66
:1075E00032484030006903221204616811400843A8
:1075F0002E494031086100BF012F05D12B48806B17
:10760000890588432949886300BF2078C007C00FD7
:10761000002809D025484030C06880088000A16853
:10762000084322494031C8600221206808400228EE
:1076300009D11E484030C0680C218843E1680843E6
:107640001A494031C86004212068084004280AD142
:1076500016484030C06803218902884321690843E5
:1076600012494031C86008212068084008280AD122
:107670000E484030C068032109038843616908430C
:107680000A494031C86080212068084080280AD11A
:1076900006484030C068032189048843A169084333
:1076A00002494031C860002020E70000001002407D
:1076B0000070004088130000F8B504460D46002C09
:1076C00001D10120F8BD79480068C007C00FA84269
:1076D0000ED276480068400840002843734908608D
:1076E00008460068C007C00FA84201D00120E9E7A2
:1076F000022120680840022807D16D48C068F021A7
:107700008843A16808436A49C8602078C007C00F51
:1077100000284CD06068022809D165480068012122
:1077200049040840400C002824D10120CAE76068C1
:10773000032809D15E480068012149060840400E2F
:10774000002817D10120BDE76068012808D15848FA
:10775000006804210840800800280BD10120B1E70F
:1077600053480068012149020840400A002801D11D
:107770000120A7E74E48C068800880006168084380
:107780004B49C860FFF7BAFB0646606802280FD174
:1077900007E0FFF7B3FB801B4649884201D903206D
:1077A00090E74348C0680C2108400828F1D134E034
:1077B000606803280FD107E0FFF7A0FB801B3D495D
:1077C000884201D903207DE73948C0680C21084070
:1077D0000C28F1D121E0606801280FD107E0FFF704
:1077E0008DFB801B3349884201D903206AE730486A
:1077F000C0680C2108400428F1D10EE007E0FFF733
:107800007DFB801B2B49884201D903205AE7284879
:10781000C0680C2108400028F1D124480068C00746
:10782000C00FA8420ED921480068400840002843F4
:107830001E49086008460068C007C00FA84201D072
:1078400001203FE7042120680840042808D1184897
:10785000C068072109028843E16808431449C860E9
:10786000082120680840082809D11148C06807216C
:10787000C90288432169C90008430D49C86000F066
:1078800049F80B49C968F022114009090A4A515CBC
:10789000C8400A4908600020FFF754FB0746002F44
:1078A00001D038460EE700200CE70000002002401F
:1078B000001002408813000042BE0008840100202E
:1078C00001480068704700008401002000B5FFF700
:1078D000F7FF0549C968072212021140090A034A45
:1078E000515CC84000BD00000010024052BE0008BC
:1078F00000B5FFF7E5FF0549C9680722D20211402C
:10790000C90A034A515CC84000BD00000010024093
:1079100052BE0008FEB52E48C7680C20384000282B
:1079200045D0042804D008280CD00C283ED10BE008
:107930002748006810210840002801D0254C00E0AD
:10794000254C41E0254C3FE00F2080043840800C5E
:1079500023490E5C032080053840800D401C0190B7
:107960001B48C068012109040840002807D01B49B2
:10797000714308460199FDF7BBFB054614E0144826
:10798000006810210840002807D0124971430846BA
:107990000199FDF7ADFB054606E00F497143084626
:1079A0000199FDF7A5FB05462C460DE000BF0848F0
:1079B0004068072149030840400B00900098401C94
:1079C00001218140CC0300BF00BF2046FEBD000066
:1079D0000010024000093D000024F40000127A006B
:1079E0005ABE0008FEB50446002C01D10120FEBDA0
:1079F000F848C6680C210E40C768012109040F40F1
:107A00002078C007C00F002872D0082E04D00C2E9A
:107A10000FD1084687420CD1EE4800680121490485
:107A20000840400C002863D06068002860D1012025
:107A3000DDE700BF012109046068884205D1E548FF
:107A400000680843E349086027E0052109046068ED
:107A500088420ED1DF480068012189040843DD49CE
:107A6000086008460068012109040843D9490860F4
:107A700013E0D8480068012109048843D54908600B
:107A800008460068012109040840009000BFD14861
:107A9000006889008843CF49086000BF60680028FB
:107AA00013D0FFF72BFA054606E0FFF727FA401B35
:107AB000642801D903209AE7C648006801214904D7
:107AC0000840400C0028F0D012E0FFF717FA0546F6
:107AD00006E0FFF713FA401B642801D9032086E76C
:107AE000BC480068012149040840400C0028F0D13E
:107AF00002212068084002287AD1E0680290042E12
:107B000003D00C2E34D1002F32D1B24800680421AA
:107B100008408008002804D00298002801D10120E4
:107B200065E7AC4840681F210902884321690902C2
:107B30000843A8494860084600680921884302991B
:107B40000843A4490860FFF7E5FEA249C968F0228E
:107B500011400909A04A515CC840A04908600020B2
:107B6000FFF7F0F901900198002841D001983EE715
:107B70000298002824D09748006809218843029978
:107B8000084394490860FFF7B9F9054606E0FFF796
:107B9000B5F9401B022801D9032028E78D48006869
:107BA0000421084080080028F1D08A4840681F213D
:107BB000090288432169090208438649486017E0A1
:107BC000844800684008400082490860FFF796F941
:107BD000054606E0FFF792F9401B022801D9032071
:107BE00005E77C4800680421084080080028F1D19E
:107BF000102120680840102867D1002E36D1754822
:107C0000006849010840400A002804D0A069002803
:107C100001D10120EBE66F48406807214903884302
:107C2000216A08436B494860084640680002000A20
:107C3000217F0906084367494860206A400B401CC1
:107C400001218140C8036349C968F0221140090934
:107C5000614A515CC840614908600020FFF772F931
:107C60000190019800284BD00198C0E6A069002837
:107C70002CD058480068FF2101310843554908605D
:107C8000FFF73CF9054606E0FFF738F9401B0228EC
:107C900001D90320ABE64F480068012149020840A2
:107CA000400A0028F0D04B48406807214903884328
:107CB000216A084347494860084640680002000AB4
:107CC000217F090608434349486019E0414800689C
:107CD000FF21013188433F490860FFF70FF905464E
:107CE00006E0FFF70BF9401B022801D903207EE6CE
:107CF00038480068012149020840400A0028F0D1B4
:107D0000082120680840082839D1606900281BD064
:107D1000304840300069012108432E494031086154
:107D2000FFF7ECF8054606E0FFF7E8F8401B0228ED
:107D300001D903205BE62748403000690221084052
:107D400040080028F0D01AE022484030006940087E
:107D50004000204940310861FFF7D0F8054606E0B1
:107D6000FFF7CCF8401B022801D903203FE6194851
:107D7000403000690221084040080028F0D1042169
:107D800020680840042879D1002000901148806BB9
:107D900089060840002806D10E48806B08430D492B
:107DA0008863012000900E480068FF2101310840DF
:107DB00000281ED10A480068084309490860FFF7F7
:107DC0009DF805460EE0FFF799F8401B642809D995
:107DD00003200CE60010024042BE0008840100208F
:107DE0000070004085480068FF21013108400028EC
:107DF000E9D000BFFF210131A068884205D1804849
:107E0000006908437E49086130E0A06800280DD170
:107E10007B480069FF2101318843794908610846A0
:107E2000006909158843764908611FE005210902A8
:107E3000A06888420DD17248006901218902084377
:107E40006F49086108460069891508436C49086153
:107E50000CE06B480069FF210131884368490861E3
:107E600008460069091588436549086100BFA06894
:107E7000002815D0FFF742F8054608E031E0FFF78B
:107E80003DF8401B5F49884201D90320AFE55C48BB
:107E90000069012149020840400A0028EFD013E0A0
:107EA000FFF72CF8054607E0FFF728F8401B554977
:107EB000884201D903209AE551480069012149020D
:107EC0000840400A0028EFD10098012808D14C480A
:107ED0004038806B0121090788434949403988634C
:107EE00000BF606A00284CD00C2E69D0606A02285E
:107EF00048D1434840380068012109068843404979
:107F000040390860FEF7FAFF054606E0FEF7F6FF87
:107F1000401B022801D9032069E539484038006830
:107F2000012149060840400E0028EFD1E16AA06A0D
:107F30000843216B084332494039C968FD221204C5
:107F4000914308432E494039C86008460068012122
:107F5000090608432A4940390860FEF7CFFF054665
:107F600006E0FEF7CBFF401B022801D903203EE5C7
:107F7000234840380068012149060840400E002887
:107F8000EFD038E01E4840380068012109068843D8
:107F90001B4940390860FEF7B1FF054606E0FEF7D1
:107FA000ADFF401B022801D9032020E514484038CA
:107FB0000068012149060840400E0028EFD11AE070
:107FC000606A012800D112E50D484038C7680120D9
:107FD00000043840A16A88420BD10F208004384049
:107FE000E16A884205D1032080053840216B884230
:107FF00001D00120FBE40020F9E400000070004003
:10800000401002408813000010B50446002C01D136
:10801000012010BD606A002800D100BF0021A162CC
:108020005120005D002804D150200155204600F069
:1080300035F802215120015520680068402188430D
:1080400021680860A16860680843E1680843216905
:1080500008436169084301225202A16911400843A3
:10806000E1690843216A0843A16A0843216808605E
:10807000A069000C04210840616A08432168486037
:108080002068C069910088432168C861002060654C
:108090000121512001550020BBE7000010B586B03A
:1080A0000446142101A8FDF796F814492068884277
:1080B00022D11348406B891408431149486300BF1B
:1080C0000846C06A012108430D49C8620846C06AD3
:1080D000C007C00F009000BF00BFE0200190022049
:1080E000029000200390032004900020059001A935
:1080F00005200007FEF7FCFD06B010BD0030014072
:108100000010024070B504462546681E09498842A1
:1081100001D901200CE0681E074948610321081FAE
:1081200000F0CAFF00200449886107200861002090
:1081300070BD0000FFFFFF0000E000E070477047E7
:10814000FEB504462068C56920680668206887680F
:108150002807000F0190019800280ED12020284008
:1081600000280AD020203040002806D0206E0028A9
:1081700002D02046216E8847FEBD019800287DD0A0
:10818000F807C00F002804D1FF202130304000281C
:10819000F5D0E807C00F00280BD0FF200130304099
:1081A000002806D0012021680862E06F0121084301
:1081B000E0670220284000280AD0F807C00F0028F6
:1081C00006D0022021680862E06F04210843E067BE
:1081D0000420284000280AD0F807C00F002806D045
:1081E000042021680862E06F02210843E06708204C
:1081F000284000280ED020203040002803D1F80766
:10820000C00F002806D0082021680862E06F08210E
:108210000843E067E06F002846D02020284000286F
:1082200009D020203040002805D0206E002802D040
:108230002046216E8847E06F0090206880684021CA
:108240000840402804D0082100980840002826D083
:10825000204602F008F92068806840210840402844
:1082600019D120688068884321688860E06E002802
:108270000DD02548E16E8863E06E00E015E0FEF762
:108280000DFB002810D0E06E816B88470CE0204683
:10829000FFF755FF08E02046FFF751FF04E02046B6
:1082A000FFF74DFF0020E06766E70120000528404A
:1082B00000280CD0012080053840002807D001207C
:1082C0000005216808622046FFF738FF54E7802048
:1082D000284000280AD080203040002806D0606E58
:1082E000002802D02046616E884745E7402028409C
:1082F000002807D040203040002803D0204602F05C
:10830000C4F839E700BF37E7A5A3000810B5044655
:10831000002C01D1012010BDA069002800D000E090
:1083200000BF606F002805D1002170200155204654
:1083300000F02CF8242060672068006840084000A6
:1083400021680860204602F007F9012800D1E2E721
:10835000606A002802D0204601F096FE206840683E
:108360000921C902884321684860206880682A2161
:1083700088432168886020680068012108432168DB
:108380000860204601F0F8FEC5E7000010B586B091
:108390000446142101A8FCF71EFF3E4920688842CC
:1083A00075D13D48406B0121890308433A49486330
:1083B00000BF0846C06A012108433749C862084621
:1083C000C06AC007C00F009000BF00BF48150190F1
:1083D00002200290002003900320049004200590C6
:1083E00001A905200007FEF783FC0120800201900F
:1083F00002200290012003900320049004200590A5
:1084000001A905200007FEF773FC244824490860F1
:1084100003204860002122488160C1608021016101
:108420000021416181612021C16109020162FEF7E1
:10843000E7FA002801D0FDF71FFC00BF1848E066EE
:10844000846200BF1548143816490860032048604C
:108450001021144881600021C16080210161002148
:1084600041618161C1610162FEF7CAFA002801D051
:10847000FDF702FC00BF0B48A066846200BF00222B
:1084800001211B20FEF7A6FF1B20FEF797FF06B079
:1084900010BD0000003801400010024030000240D2
:1084A00090170020D817002070B504460D461646D8
:1084B000A06F202863D1002D01D0002E01D1012012
:1084C00070BD01210903A068884208D120690028F5
:1084D00005D1E807C00F002801D00120F0E700BF58
:1084E0007020005D012801D10220E9E70121702000
:1084F000015500BF6565582006530020E067222023
:10850000A067E06E002820D01E48E16EC8621E48B9
:10851000E16E08631D48E16E48630020E16E8863E8
:108520002368194624313346626DE06EFEF7BCFACB
:1085300000280AD01020E06700BF002170200155FC
:1085400000BF202060670120BAE700BF0021702033
:10855000015500BF20680068FF21013108432168F0
:1085600008602068806801210843216888602068CD
:10857000806840210843216888600020A0E702202D
:108580009EE700000FA4000859A40008BDA300083E
:1085900070477047FFB583B004460D461746606FBD
:1085A000202875D1002D01D0002F02D1012007B065
:1085B000F0BD01210903A068884208D12069002884
:1085C00005D1E807C00F002801D00120EFE700BF68
:1085D0007020005D012801D10220E8E70121702010
:1085E000015500BF0020E06721206067FEF786FC90
:1085F0000190502007535220075301210903A0681E
:10860000884205D12069002802D10026029502E0A7
:108610002E460020029021E0069800900022802142
:108620002046019B02F086F9002801D00320BEE716
:10863000002E09D102980088C005C00D216888620B
:108640000298801C029003E0307821688862761CD2
:108650005220005B401E81B2522001535220005B29
:108660000028D9D106980090002240212046019B85
:1086700002F060F9002801D0032098E7202060670D
:1086800000BF00217020015500BF00208FE7FFE7E9
:1086900002208CE7704700BFFEE710B500220421DE
:1086A00005200007FEF723FC002208210520000713
:1086B000FEF71DFC0A2002F0E3FC01220421052044
:1086C0000007FEF714FC0A2002F0DAFC0022042165
:1086D00005200007FEF70BFC10BD10B50022042199
:1086E00005200007FEF703FC0122082105200007F2
:1086F000FEF7FDFB0A2002F0C3FC01220421052045
:108700000007FEF7F4FB0A2002F0BAFC0022042165
:1087100005200007FEF7EBFB10BD70B505460024F1
:1087200000261EE00022042105200007FEF7DFFBE3
:108730000A2002F0A5FC0122042105200007FEF713
:10874000D6FB6006040E082105200007FEF7C6FBD5
:10875000002801D0601CC4B2052002F091FC701CFE
:10876000C6B2082EDEDB002D02D1FFF7B6FF01E016
:10877000FFF793FF204670BD70B504460022042128
:1087800005200007FEF7B3FB00252AE080202040EB
:10879000C011002806D00122082105200007FEF79D
:1087A000A6FB05E00022082105200007FEF79FFB3D
:1087B0006006040E0A2002F063FC01220421052059
:1087C0000007FEF794FB0A2002F05AFC0022042165
:1087D00005200007FEF78BFB0A2002F051FC681C05
:1087E000C5B2082DD2DB70BD10B5012208210520CD
:1087F0000007FEF77CFB0122042105200007FEF79D
:1088000076FB0022082105200007FEF770FB0A20F6
:1088100002F036FC0022042105200007FEF767FB6A
:1088200010BD10B50022042105200007FEF75FFBF4
:108830000022082105200007FEF759FB0A2002F05C
:108840001FFC0122042105200007FEF750FB012236
:10885000082105200007FEF74AFB0A2002F010FC61
:1088600010BD10B500240122082105200007FEF7E5
:108870003EFB062002F004FC012204210520000733
:10888000FEF735FB062002F0FBFB07E0601CC4B2DC
:10889000FA2C03DDFFF7C5FF012010BD08210520DC
:1088A0000007FEF71BFB0028F0D100220421052061
:1088B0000007FEF71CFB0020EFE7000038B501F0D1
:1088C00093FC01F0E5FC6D480068C0690221084096
:1088D000002802D06A486B49C860FDF71FFB0446B8
:1088E00069484088002808DD67484088401E81B2FA
:1088F0006548418001206549087064480078002877
:1089000006D001280AD0022817D0032822D11BE064
:10891000012291025E48FEF7EAFA1BE0212C06DAFA
:108920000022012189025A48FEF7E1FA04E00122FF
:1089300091025748FEF7DBFA0CE000220121890280
:108940005348FEF7D4FA05E0012291025048FEF7A1
:10895000CEFA00BF00BF0121C9024D48FEF7BEFAA2
:10896000002825D04B480078002804D1012049492F
:10897000087002F027F84848007863280BDD0022D1
:1089800008214348FEF7B3FA0122D103052000076E
:10899000FEF7ADFA1BE0012208213D48FEF7A7FAD9
:1089A00000220121C90305200007FEF7A0FA0EE00E
:1089B000002038490870002208213548FEF797FA50
:1089C00000220121C90305200007FEF790FA2E4876
:1089D000808C012820D100253048009072B680217B
:1089E0002F48FDF765F90546002D05D0022269469E
:1089F0002B48FDF74FFA054662B62AA002F0EEF8C2
:108A000000212148818403F08BF9642002F02EFBC1
:108A10001B481C49C86000BF1B48408C01280ED170
:108A2000002119484184002017494039088003F08B
:108A300077F9642002F01AFB11481249C860124805
:108A4000008C01280AD100210F48018403F068F945
:108A5000642002F00BFB0A480A49C8600A48403803
:108A600000881449884204D107484038C08800284B
:108A700002D103480349C86038BD00001017002028
:108A80000400FA0500ED00E0F80D0020360100209A
:108A900000040050640100204C010020AAAA00003C
:108AA000384A0008BDF8C8EBC9FDBCB6C4A3CABDAE
:108AB0000D0A0000AA55000008B53721202000F05B
:108AC00077F80321212000F073F84021222000F0E4
:108AD0006FF80821232000F06BF8AA21302000F065
:108AE00067F802200B4908870846008FC1B2322080
:108AF00000F05EF80121332000F05AF85F212020B9
:108B000000F056F8684600F007F80A2002F0B8FABC
:108B100008BD0000B80D002010B5044621460F2006
:108B200000F023F8002800D110BD0120FCE770B54B
:108B300004460025FFF758FE3220FFF71DFEFFF721
:108B400090FEE0B2FFF718FEFFF78BFEFFF74CFE3A
:108B50003320FFF711FEFFF784FE0020FFF7DDFD55
:108B60000546FFF75EFE284670BD70B505460C460B
:108B70002846FFF7DCFF2070012070BD70B5044669
:108B80000D46FFF731FE3220FFF7F6FDFFF769FED5
:108B9000E0B2FFF7F1FDFFF764FE2846FFF7ECFDBA
:108BA000FFF75FFEFFF73DFE0A2002F069FA70BD95
:108BB00070B504460D4629462046FFF7DFFF012029
:108BC00070BD000010B50248FEF78FFA10BD00001E
:108BD00088160020F0B585B004460020039072B6D8
:108BE0004F4920684018002806D14E48C06803212C
:108BF00089040840039000E000BF00BF206880683F
:108C000002902068C06801902068456920688669E4
:108C100043492068401800280DD142484038806AF6
:108C2000490508433F49403988620846806A400048
:108C30004008886200E000BF00BF002D01D1002E77
:108C40005FD0374920684018002807D13548C068F0
:108C50000321890488433349C86000E000BF00BF96
:108C6000002D1DD02068006901210843216808619A
:108C700020684561FEF742F9074600BFFEF73EF95E
:108C8000C01B00902068006808210840082804D014
:108C90007D21C90000988842F0D9082021684860E9
:108CA000002E1DD020680069012108432168086159
:108CB00020688661FEF722F9074600BFFEF71EF91D
:108CC000C01B00902068006810210840102804D0C4
:108CD0007D21C90000988842F0D9102021684860A1
:108CE0000F4920684018002809D10E48C0680321A8
:108CF00089048843039908430A49C86000E000BF1B
:108D000000BF20680069400840002168086102989F
:108D10002168886001982168C86062B605B0F0BD1E
:108D20000084FFBF401002401CB50020009001905D
:108D30001E481F49086000211D48C16301208007AB
:108D40001B49486000211A48816007218163012185
:108D500001610021C160001D01774177001F816220
:108D6000FF21C231416200212430017204212438E4
:108D700041610021016381614163C161FDF78EFBA7
:108D8000002801D0FCF778FF0A480090801301907A
:108D900069460748FDF7F6FA002801D0FCF76CFF9A
:108DA00000210348FDF780FA1CBD000000240140AB
:108DB0002C1600200200000408B500BF0A48006B12
:108DC00001210843084908630846006BC007C00F2B
:108DD000009000BF00BF002201210A20FEF7FAFA2E
:108DE0000A20FEF7EBFA08BD0010024000B587B07C
:108DF000142102A8FCF7EFF900BF6548C06A0421FE
:108E000008436349C8620846C06A042108400190CB
:108E100000BF00BF00BF5E48C06A802108435C49B4
:108E2000C8620846C06A80210840019000BF00BFA8
:108E300000BF5748C06A012108435549C862084627
:108E4000C06AC007C00F019000BF00BF00BF084646
:108E5000C06A022108434E49C8620846C06A02211E
:108E60000840019000BF00BF01221C21052000071F
:108E7000FEF73DF8012247494748FEF738F800223F
:108E800046494548FEF733F80022912109020520A2
:108E90000007FEF72CF801200290414803900020C3
:108EA000049002A905200007FDF722FF022002908E
:108EB000032003900020049002A905200007FDF77D
:108EC00017FF0C2002901120039000200490032033
:108ED000059002A905200007FDF70AFF1020029067
:108EE00001200390002004900220059002A9052093
:108EF0000007FDF7FDFE01200290112003900020E5
:108F00000490059002A92448FDF7F2FE0220029089
:108F1000244803900120049002A91F48FDF7E8FEB1
:108F2000214802900120039000200490059002A99E
:108F30001948FDF7DDFE0120C002029000200390D9
:108F40000220049002A91448FDF7D2FE91200002ED
:108F500002900120039000200490059002A90520B2
:108F60000007FDF7C5FE802002900020039001203D
:108F7000049002A90848FDF7BBFE0022012105204C
:108F8000FEF728FA0520FEF719FA07B000BD000029
:108F900000100240010400000004005008300000EE
:108FA00000001110000021100834000010B50A481C
:108FB0000A4908600020486000210848816008498B
:108FC00041610021016241628162FEF719F90028C6
:108FD00001D0FCF751FE10BD007C00408816002037
:108FE000FFFF000010B5124812490860FF2005304D
:108FF000486000210F488160C16001614161012129
:10900000490281610021C1610162416281620721DF
:10901000C162FEF7F9FF002801D0FCF72DFE0548DC
:10902000006800684021084302490968086010BDD3
:1090300000300140B816002000B585B01421684604
:10904000FCF7C9F819481A490860E1204002486055
:10905000002117488160C16001610C21416100213C
:109060008161C16101623020114948620121090317
:109070000F4881634900C163FFF748F9002801D018
:10908000FCF7FAFD012080020090022001900120EF
:1090900002900320039004200490694605200007F5
:1090A000FDF726FE01F088FC05B000BD0038014048
:1090B000101700207047000010B5002819DA1A4A6E
:1090C00003071B0F083B9B089B00D2588307DC0E4D
:1090D000FF23A3409A438B071B0E8407E40EA34093
:1090E0001A43114B0407240F083CA408A4001A518A
:1090F00018E00E4A03231B02D21883089B00D258A3
:109100008307DC0EFF23A3409A438B071B0E8407C3
:10911000E40EA3401A43054B032424021B198408C0
:10912000A4001A5110BD00001CED00E000E100E0B9
:1091300000BF00BF00BFBFF34F8F00BF00BF00BF25
:1091400006480749C86000BF00BF00BFBFF34F8F8C
:1091500000BF00BF00BF00BF00BFFDE70400FA056D
:1091600000ED00E0F0B593B000200E90962002F0E4
:10917000F1FA4B20C00002F009FB0020FE49087004
:10918000FE4800780C2802DB0B20FC490870012205
:10919000510205200007FDF7AAFEF8480078F849BB
:1091A0000870F6480078F74908700020F649087002
:1091B000F6490870F6480078F64908710221F64829
:1091C000FDF78CFE002801D1012000E00020F349CA
:1091D000097849000843EF49C871F14801780068EF
:1091E000401CEF4A1060C8B2EA49C870E5480078F0
:1091F0008872E44800784200EA49E6480B30FBF701
:10920000D1FF0620E34948720846E7490A784270D0
:1092100049788170DB490978490008460D30002201
:10922000DC4902F0B5FBD7490978490008460D3002
:10923000002102F0C1FB022002F0E6FA0020D5492D
:10924000C871DA490870DA4908700120D9490870F4
:109250000020D9490870D948FEF75EF8D84908803F
:109260000020C9490870C7480078FCF700FA064694
:10927000FCF77CFAD34AD44B05910490FCF70CF927
:109280000791069001F08EFE0022D04B09910890C4
:10929000FCF750F80B910A90FCF74AFAC0B20D9017
:1092A0000D984001C64909884018C94908800846F8
:1092B00000880121C903884204DBC5480088401AA0
:1092C000C3490880C348C4490860C4480078401CAA
:1092D000C2490870B948FEF71FF8C1490880AFE2DB
:1092E000B648FEF719F8BE49088033E0B048007868
:1092F00000281BD002F0EAF91090129910988842C9
:1093000014D911991098884210D202F06BF80020FD
:10931000A8490870384602F015FA012002F074FAE4
:10932000B04908700020A24908701DE0A348FDF76D
:10933000F3FFAB49088008460088A54909888842A0
:1093400008DBA7480088A2490988A74A89188842EB
:1093500000DA09E000210F2002F054F9A349086067
:10936000A34908400028C1D000BFA0480068401CA5
:10937000002801D1FFF7DCFE9C4800680121890329
:10938000084000287ED08122D20100210F2002F067
:10939000B8FA0021102002F035F94006400E0F9077
:1093A000002294480F9902F07DF9002002F0EEF9B6
:1093B000002002F09AF98F48407A07288FD10222C4
:1093C0008D498C48401DFBF711FF002887D102F022
:1093D00050FB8A4A03C202F035FB894A03C26A483D
:1093E0000078401C684908708248427808A90A74CD
:1093F0008078487462480078002810D101208149A3
:1094000008706846008E6749088001205D49087031
:10941000604908A8007C487008A8407C88706148B2
:1094200000886946098E88427ED177497148C08993
:10943000088076486F49098A01806048FDF76CFF13
:109440006749088071480088FF30C3306F49088041
:10945000084600886E49884212DD6C480088401A30
:109460006A49088068480088401C674908800846A7
:10947000008867490B31884202DB0020624908807E
:10948000002600E0D0E1032062498855624959482E
:1094900042890A808089488008460068B1005F4A96
:1094A00050505448C07C0007000F032805D0514895
:1094B000C07C0007000F354908704E48C07C001181
:1094C0005749087000204549087001203849087044
:1094D0004149484842890A80808948802948007863
:1094E000FF2191314843FF309B30FF30F5300004BD
:1094F000C117434B0CCB801859410906070A0F438B
:109500004848381A129019208002381811907908AA
:10951000490000200A0E000210430B0200221146EF
:109520009A184841404900E006E10A604860334823
:109530000CC818480A3002F06BFA31480CC81548BC
:10954000163002F065FA38480CC81248123002F0A2
:109550005FFA08200F49487231480078002871D01E
:10956000022225492348401DFBF740FE002869D10F
:1095700001200E49087059E0E90000202A0100206E
:1095800029010020280100200901002036010020C7
:109590004C0100202C120020000400502E0100205D
:1095A0006C00002026140020020100202C01002065
:1095B0001C0100201E0100201D0100208816002033
:1095C00022010020666666666666E63F0000084087
:1095D00024010020A08601000401002019010020C0
:1095E00020010020E8000020983A000070000020D0
:1095F00000D027247C1200204001002078000020A9
:10960000800000201B01002048010020F400002001
:10961000E7030000E8140020F800002058140020A0
:10962000370100200052030088000020FD49C87166
:109630000F981638FC49087008460278FB49FC4828
:10964000FBF7B0FDFB490978890008461C30002271
:10965000F44902F09DF9F7490978890008461C3061
:10966000002102F0A9F90120F34908700422EF4912
:109670001339F248FBF796FDF14800887D21C900B7
:109680004843F04909884018EF490860EF480078DE
:10969000EF490870EF49C888FBF7E9FF0990E848EF
:1096A0000088FBF7E4FF08900999FBF705FE7F218E
:1096B000C9050A90FBF7A7FD0B90FCF701F8E349F9
:1096C0000880E3480078401E0988884202D10120C2
:1096D000D9490870DA480088DF490880DF4900204E
:1096E000085EFBF7CBFF09910890DD480088FBF787
:1096F000D9FFDC4ADC4B01910090FBF7CDFE0591D0
:109700000490D1480068FBF7B9FF03910290059BD4
:10971000049AFBF7B3FE07910690099B089AFBF7A2
:1097200009FE0B910A90FBF7DFFFD0490860D04893
:10973000008800F091FB76E06846008EFCF7D8FBCD
:109740000646CC4909788E4213DB0120CA490870CD
:10975000B8480078401CB74908706846008E710010
:10976000C64A5052AF4908A8007C487008A8407CFF
:1097700088700320C2498855C249AC4814384289D0
:109780000A808089488008460068B100BE4A50506F
:10979000A6481438C07C0007000FBC4909788842ED
:1097A0000BDDA2481438C07C0007000F032804D04A
:1097B0009E481438C07CB5490870B5480078002828
:1097C00016D00222B34999480F38FBF70FFD002845
:1097D0000ED10120B04908709249C8710F9816380F
:1097E000914908700846027890499148FBF7DAFCE5
:1097F000B00016308B4940180B90A8480CC80B9845
:1098000002F006F98B490978890008461C300022CD
:10981000844902F0BDF887490978890008461C3060
:10982000002102F0C9F80BE09D4A00210F2002F050
:1098300068F89C480078002802D0002001F055FF0D
:109840008748008898490988884200DA48E58448B2
:10985000008895490988954A89188842F6DC904A1B
:1098600000210F2002F04DF89148007871490870EE
:10987000002583480078002818D170480068FCF75C
:1098800023FC8C49088008880988491E894B198067
:1098900089490988FBF742FC88480088414388B21F
:1098A000734908800846008800F0D6FA00208449F1
:1098B0000870002423E07248005D00281DDD804808
:1098C0000078401C7E4908706D48005DA9007D4A03
:1098D000505060006949085A69007B4A5052A00004
:1098E00069490A582946681CC5B2880077490A5058
:1098F0006348005D401E62490855601CC4B25D4863
:1099000000785D4909784018A042D4DC68480078A6
:10991000032803DA6A4800786949087068480078C3
:109920005449087000243FE0002536E0A80067494C
:109930000958681C8000654A105881422BDDAA0036
:10994000624B99586A00604B985AA2005D4B9A5836
:109950000C926A1C92005D4B9A58AB005B4EF25021
:109960006A1C5200584B9A5A6B00574EF2526A1CAE
:109970009200544B9A58AB00524EF2506A1C92001F
:10998000524B99506A1C52004F4B98526B1C9B00D3
:109990000C9AF25000BF681CC5B236480078401ED1
:1099A000A842C3DC601CC4B232480078401EA0420A
:1099B000BADC002046490870002496E06000424965
:1099C000085A61002D4A5052A00040490858A10091
:1099D0002D4A5050A000114608583E4988427DD07B
:1099E000A000384908580A287DD139480078062156
:1099F0004843001D384940186100204A89180A78F8
:109A0000027049784170A2001F4BD118304A127879
:109A100006235A43921D304BD0180422FBF7C2FB99
:109A20002B485CE02C1200202D0100209012002019
:109A3000F4140020280100201D0100203001002026
:109A400048010020F40000200C01002068010020E3
:109A50002B010020B80D0020260100203401002039
:109A600020010020F853E3A59B843E401401002010
:109A70004E010020290100201B0100202614002097
:109A8000E8140020F80000205814002036010020BF
:109A900037010020400100202C0100208000002020
:109AA00000D027241E01002024010020983A000045
:109AB00009010020FC000020540100205201002078
:109AC0002A010020B81400203E1400208814002031
:109AD0001A010020FFFF0100DA13002003E00078E4
:109AE000401C21490870601CC4B2204800788442A0
:109AF00000DA63E7002405E01D48A1001D4A50502C
:109B0000601CC4B20C2CF7DB1B48007800281CD06A
:109B100000200C9000260B90184800780B901748F6
:109B2000467880780C900B9802280DD1144988193A
:109B30001249C91C0C9AFBF735FB02F0F1F86420BE
:109B400001F094FAFFF7F4FA00BF0E4A00210F204B
:109B500001F0D7FE00220121490205200007FDF790
:109B6000C6F913B0F0BD00001A0100202901002041
:109B7000FFFF0100581400202C010020F4140020E5
:109B8000B80D002080D0272470470000F0B585B0C4
:109B900051485249086002F04FF8FF2011305049F7
:109BA00048800846C088002801D16420C8804D48FC
:109BB0000078432802DD43204A490870494800786C
:109BC000002802DA0020474908704548C08E454900
:109BD00008704348C08F444908704148808F43490A
:109BE00008703F48807A424908703D488088414962
:109BF00008603B490889FBF755FD04463E4A3F4B48
:109C0000FBF74AFC0191009001F0CCF906460022D6
:109C10003B4BFBF78FFB03910290FBF789FD394922
:109C200008802F49C88837490988FBF777FA3649F1
:109C300008802B49888834490988FBF76FFA314836
:109C40000088414388B23149088009887D22D200CA
:109C500051430846FBF712FD06462D4A2D4BFBF7F4
:109C600083FC0446FBF764FD2B49088027480088E5
:109C70002A4908801A48C1887D20C000FBF74EFAA7
:109C8000274908801648C1887D20C000FBF746FAA6
:109C900024490880012024490880FCF73FF9234922
:109CA00008801D48028822492248FDF739FB002818
:109CB00001D0FBF7E1FF0F4801681FA000F08EFF05
:109CC0000748C18820A000F089FF0548018923A02A
:109CD00000F084FF05B0F0BD01AA00084800002094
:109CE000B80D002001000020620100206301002067
:109CF0004B01002040010020666666666666E63F0E
:109D00000000084052010020540100204E010020B4
:109D1000F853E3A59B843E405A0100205E010020D9
:109D20005C01002066010020680100206001002025
:109D3000FF7F000088160020B1EAC7A949443A20F5
:109D40002564202E0D0A0000CDA8D1B6BCE4B8F4DD
:109D50003A202564206D732E0D0A0000B5A5B4CEFF
:109D6000CDA8D1B6BBF9D5BECAFDC1BF3A20256486
:109D7000B8F62E0D0A00000000B585B01421684623
:109D8000FBF729FA00220121C9031048FDF7AFF8BB
:109D90000120C00300900120019000200290039058
:109DA00069460A48FCF7A4FF0120C0030090032085
:109DB000019000200290039069460448FCF798FF48
:109DC000022001F053F905B000BD0000000400506E
:109DD0007047000038B504460D460020009055201D
:109DE0001B490870AA20487003208870601DC87045
:109DF000032008710846457184716800154A81186E
:109E000022461348C01DFBF7CDF9002008E0811C55
:109E10000F4A525C6946098851188AB20092401C68
:109E2000611D8842F3DB0A48801CFBF771FE00903D
:109E3000E01D074941186846007808706846407878
:109E4000487021460931024800F038FB38BD000057
:109E5000C8150020B80D0020F0B585B005461A4899
:109E600000881A490988884206DB17480088174984
:109E70000988401A144908801548C0881249098881
:109E8000484347197D21C9004F43124800683E1AD4
:109E90003046FBF7F3FB104A104B01910090FBF7A3
:109EA00063FB03910290FBF71FFC04460C498C42B4
:109EB00001DD0846241A002C01DA09482418094853
:109EC0000068446105B0F0BD680100206601002013
:109ED000B80D002014010020F853E3A59B843E40F8
:109EE000FF7F00008816002001460020054A126806
:109EF00090B2054A104002460A431046014A1060DB
:109F00007047000000300140C7FF000010B5FCF7AB
:109F1000FBFF10BD00B599B034210CA8FBF75BF92D
:109F2000142107A8FBF757F91C216846FBF753F9E2
:109F3000244800680321C90288430121C90240184E
:109F400020490860FDF758FA1F4800690321C9023B
:109F500088431D49086106200C9088150E90012049
:109F60000F901020109002201590002116914104AE
:109F70001791410518910CA8FDF734FD002801D078
:109F8000FBF77AFE0F20079003200890002009902D
:109F90000A900B90012107A8FDF78EFB002801D045
:109FA000FBF76AFE812000900020029003208004CD
:109FB00006906846FDF76AFA002801D0FBF75CFEC0
:109FC00019B000BD00700040401002401548006804
:109FD000FF2101310843134908600846C06812494F
:109FE00008401049C86008460068104908400D49FB
:109FF000086008468068400840008860084600689D
:10A00000012189048843074908600846C068FD218A
:10A01000090488430349C8600020086104480549D1
:10A0200088607047001002400C40FF88F6FFF6FE83
:10A030000050000800ED00E010B501F0FDFA044604
:10A0400002E001F0F9FA04460C488442F9D10020FC
:10A050000B4908800B480078002804D0012803D061
:10A06000022807D103E005E0FBF77AFF02E0FFF7E3
:10A0700079F800BF00BF01F099F910BD3001CADEC8
:10A08000E600002060000020818CC907C90F00296C
:10A0900008D001684968012252049143826A114341
:10A0A000026851600222416A1140022907D1016809
:10A0B0004968D2039143C26A114302685160042285
:10A0C000416A1140042907D101684968120491438B
:10A0D000026B1143026851600822416A114008294D
:10A0E00007D10168496812039143426B114302682A
:10A0F00051601022416A1140102907D10168896816
:10A1000012029143826B1143026891602022416ADE
:10A110001140202907D10168896812029143C26B5E
:10A120001143026891604022416A1140402915D1D3
:10A130000168496892039143026C114302685160BF
:10A1400001221205016C914208D10168496803227D
:10A1500052059143426C1143026851608022416A6A
:10A160001140802907D10168496812039143826C2C
:10A17000114302685160704738B504460020E0671B
:10A18000FCF7BCFE05462068006808210840082846
:10A190000BD114482B46002289040090204600F081
:10A1A000C9FB002801D0032038BD206800680421C5
:10A1B000084004280BD10B482B46002209050090CB
:10A1C000204600F0B7FB002801D00320ECE7202058
:10A1D0006067A06700BF00217020015500BF00200C
:10A1E000E2E70000FFFFFF0170B50025C82420480A
:10A1F0000078002800D070BD1E480078002800D0EC
:10A20000F9E701201B4908701B48406B002801D169
:10A210000870F0E71848406BC8210D1A1CE0174978
:10A22000174A1268885C17490968884716480088E9
:10A230000A2148431549088011480068401C10490C
:10A24000086008460068C82801DB002008600A484A
:10A25000406BC8210D1A641E09480068A84201D04D
:10A26000002CDCDC00200349087000BFC3E70000BD
:10A27000420000204400002000000240F00C0020BA
:10A2800038000020480000205C0100207001002000
:10A2900010B53A480078002803D1394800780028E2
:10A2A00000D010BD0120364908703648C0698021B1
:10A2B0000840002802D132490870F2E732490020F4
:10A2C0000856324900228A56904215D12D48C0695D
:10A2D0004021084000280BD02D480078002807D0E6
:10A2E00000202B4908702B480088401C2949088011
:10A2F000002023490870D4E725480078002805D1BC
:10A300000120234908700A2000F0BAFE1F490020EE
:10A310000856CC21484320494018001D1F490968B0
:10A32000405C184988621D480068401C1B49086051
:10A33000164900200856CC214843174908581749A8
:10A340000968884214DC0020144908600F4800782E
:10A35000401C40B20D490870084600780E2801D113
:10A36000002008700E480078401C40B20C4908706C
:10A3700000200349087000BF93E70000420000205E
:10A380004300002000380140350000203400002048
:10A390004500002052000020C80100205800002085
:10A3A0003600002070B50546AC6A00215A200153E2
:10A3B000522001532046FDF7C2FE70BDF8B5054698
:10A3C000AC6A666FA76F206880688021084080288B
:10A3D00007D1212E05D1002152200153204600F043
:10A3E00064F82068806840210840402807D1222F67
:10A3F00005D100215A200153204600F034F8E06FC7
:10A4000010210843E0672046FDF799FEF8BD70B5BE
:10A410000546AC6A2868006820210840002817D14A
:10A4200000215A20015320680068FF210131884330
:10A4300021680860206880684008400021688860C2
:10A440002068806840218843216888602020A067B8
:10A450002046FEF79DF870BD70B50446A56A2846F3
:10A46000FEF797F870BD01680968FF222132914319
:10A4700002681160016889684908490002689160B2
:10A480002021816700210166704710B504462068CD
:10A490000068402188432168086020206067002010
:10A4A00060662046FEF7F6F810BD01680968C02214
:10A4B00091430268116020214167704770B50546DD
:10A4C0000C4620480078002803D11F480078002857
:10A4D00000D070BD01201B490870C82C04DC1B484B
:10A4E00000214156002903DC002016490870F0E7DE
:10A4F000174900200856CC21484316490C50144AED
:10A5000000215156CC225143124A8918081D224677
:10A510002946FAF747FE0E480078401C40B20C4925
:10A520000870084600780E2801D1002008700748FE
:10A530000078401E40B205490870002001490870AB
:10A5400000BFC6E742000020430000203600002084
:10A5500035000020C8010020F0B587B00446102067
:10A5600004900025002003900026E74920688842D7
:10A5700000D100E000BF2169A06808436169084379
:10A58000E1690843074620680068E049084038430D
:10A590002168086020684068032109038843E16856
:10A5A000084321684860A769D7492068884201D0DC
:10A5B000206A0743206880680B21090288433843DA
:10A5C0002168886000BFD249206888421CD1D148E8
:10A5D000C0688007800F002806D001280AD0022812
:10A5E00005D003280CD108E0012004900BE00220E4
:10A5F000049008E00420049005E00820049002E0A4
:10A600001020049000BF46E0C349206888421CD156
:10A61000C048C0680C210840002806D004280AD091
:10A62000082805D00C280CD108E0002004900BE08D
:10A630000220049008E00420049005E00820049023
:10A6400002E01020049000BF25E0AF492068884256
:10A650001FD1B048C068032189020840002808D0F3
:10A6600001218902401A0AD0401A05D0401A0CD1A3
:10A6700008E0002004900BE00220049008E0042091
:10A68000049005E00820049002E01020049000BF30
:10A6900001E01020049000BF9B492068884256D1F9
:10A6A000049804281AD004DC002807D002281CD102
:10A6B00008E0082816D0102817D117E0FDF706F992
:10A6C000064616E09348403800681021084000090B
:10A6D000002801D0914E00E0914E0AE0FDF71AF9F2
:10A6E000064606E00126F60303E000BF01200390C2
:10A6F00000BF00BF002E0AD0606841004018B04281
:10A7000003D860680003B04202D201200390F4E055
:10A71000606802903046FF21013100F086FA6268DD
:10A72000520800238018594101910090029AFAF7CB
:10A7300009FD054603200002854205D3794885427C
:10A7400002D82068C560D8E001200390D5E001213F
:10A75000C903E06988426FD1049804283CD006DC24
:10A76000002809D0012813D002284AD11CE008286B
:10A770003ED0102845D145E0FDF7A8F840006168BB
:10A780004908401802906168FAF7B2FC85B23CE0D3
:10A79000FDF7AEF840006168490840180290616812
:10A7A000FAF7A6FC85B230E05A484038006810211C
:10A7B00008400009002807D061684A085A4BD018A1
:10A7C000FAF796FC85B206E061684A08574BD01844
:10A7D000FAF78EFC85B218E0FDF79CF8400061683E
:10A7E0004908401802906168FAF782FC85B20CE0D3
:10A7F00061684A0801231B04D018FAF779FC85B276
:10A8000003E000BF0120039000BF00BF102D0FD355
:10A81000474885420CD846480F38284005902807FD
:10A82000400F05990843059005982168C86064E0C9
:10A830000120039061E0FFE7049804283AD006DC89
:10A84000002809D0012812D0022847D11AE0082890
:10A850003BD0102842D142E0FDF738F86168490842
:10A86000401802906168FAF743FC85B23AE0FDF7C0
:10A870003FF861684908401802906168FAF738FCAF
:10A8800085B22FE0234840380068102108400009B5
:10A89000002807D061684A08204BD018FAF728FC36
:10A8A00085B206E061684A081D4BD018FAF720FC13
:10A8B00085B217E0FDF72EF861684908401802904C
:10A8C0006168FAF715FC85B20CE061684A0801235B
:10A8D000DB03D018FAF70CFC85B203E000BF0120BF
:10A8E000039000BF00BF102D05D31148854202D848
:10A8F0002068C56001E001200390002020666066AA
:10A90000039807B0F0BD000000480040F369FFEF76
:10A9100000380140401002400044004000093D0062
:10A920000024F400FFFF0F0000127A000048E80145
:10A93000FFFF0000FFB581B004460D4617460A9E92
:10A9400022E0701C00281FD0FCF7D8FA0499401AA6
:10A95000B04201D8002E17D120680068FF21A13134
:10A9600088432168086020688068400840002168AA
:10A97000886020206067A06700BF0021702001551B
:10A9800000BF032005B0F0BD2068C0692840A84280
:10A9900001D1012000E00020B842D2D00020F1E730
:10A9A00010B510200349096808620248FDF7C8FB8A
:10A9B00010BD0000101700200D20014908707047DD
:10A9C0003600002010B50A4800880A21484309498A
:10A9D0000880FEF7F1F9FEF72FFBC8220649074869
:10A9E000FDF762FD002801D0FBF746F910BD00001D
:10A9F0005C01002070010020F00C002010170020E6
:10AA000070B5044600256A480078082865D100BF63
:10AA1000002004E06749095C49198DB2401C664971
:10AA20000978491F8142F5DC64480078281885B20E
:10AA300061480078281885B261480078281885B2E6
:10AA400060480078281885B25F480078281885B2D9
:10AA50006019C007C00F002835D058480078012879
:10AA600027D002282DD15949554A127888185549BE
:10AA70000A785049FAF796FB01F052F9642000F089
:10AA8000F5FA00BF00BF00BF00BF00BFBFF34F8F8C
:10AA900000BF00BF00BF4E484E49C86000BF00BFA6
:10AAA00000BFBFF34F8F00BF00BF00BF00BF00BF9C
:10AAB000FDE743480078411042480078FFF78AF9E3
:10AAC00000E000BF00BF0020394908703C49087011
:10AAD000394908704049087068E03548007807280F
:10AAE00012D134483C49097844543B480078401C12
:10AAF0003949087030480078401F0978884255D19C
:10AB000008202B49087051E029480078062805D113
:10AB10002C48047007202649087047E02448007834
:10AB2000052805D1264804700620214908703DE01B
:10AB30001F480078042805D12048047005201C49CE
:10AB4000087033E01A480078032808D11A480470C6
:10AB500000201B49087004201549087026E014489D
:10AB60000078002805D1552C03D101201049087028
:10AB70001CE00F480078012805D1AA2C03D102203F
:10AB80000B49087012E00A480078022807D1032C0C
:10AB900005D10320064908700B48047006E0002028
:10ABA00003490870064908700349087070BD000029
:10ABB00039010020641500203B0100203E010020E7
:10ABC0003C0100203A0100203D010020B80D00208A
:10ABD0000400FA0500ED00E03F0100200FB410B5BD
:10ABE00003A9044B044A029800F034F910BC08BCD5
:10ABF00004B018472DBA0008880100202021020C5B
:10AC000001D010211046020A01D01046083902096D
:10AC100001D01046091F820801D01046891E420843
:10AC200001D0881E7047081A7047F8B582B28BB2FF
:10AC3000040C0D0C10465843002126465E43370C89
:10AC400036048019794116466E43370C3604801954
:10AC5000794126466E438919F8BD30B47446641EA6
:10AC60002578641CAB4204D3635D5B00E31830BC01
:10AC700018471D46F8E702E008C8121F08C1002A5D
:10AC8000FAD170477047002001E001C1121F002A6D
:10AC9000FBD1704708B5002100916B4601220221CB
:10ACA0002C2000F043FE022100916B4601222C2053
:10ACB00000F03CFE08BD000038B504466D20009051
:10ACC0006B46012208492E2000F030FE002C05D0F2
:10ACD000064A07492E2000F003FE04E0054A044915
:10ACE0002E2000F0FDFD38BD06080000070600001C
:10ACF000061800000716000038B504466B4602220D
:10AD00000021362000F09EFC2300FFF7A6FF0E1165
:10AD1000081A54545454233154543D444B54002184
:10AD2000684601704078FE2108406946487043E05B
:10AD300069460878FC2108400121084369460870EB
:10AD40003AE069460878FC21084002210843694638
:10AD5000087031E068460078B3210840482101437B
:10AD6000684601704078802108436946487023E0B6
:10AD700068460178B320014068460170407841067A
:10AD8000490E6846417017E0694648780221084339
:10AD90006946487010E069464878FD2108406946D8
:10ADA000487009E069460878CF210840202108430F
:10ADB0006946087000E000BF00BF6B460122002119
:10ADC000362000F0B3FD00AB0133012211463620DE
:10ADD00000F0ACFD38BD08B5032168464170012183
:10ADE00001706B4602220021362000F09FFD0122F7
:10ADF000D20306212D2000F073FD012000F036F96A
:10AE00000120FFF779FF08BD38B504462004010E84
:10AE10006846417004706B46022204212D2000F028
:10AE200085FD0321684601706B46012206212D2015
:10AE300000F07CFD0021684601706B46012206216E
:10AE40002D2000F073FD0A212D2000F0DBFB0546CC
:10AE5000284638BDFFB58DB00446002506E02528FC
:10AE60000AD0109A0F999047641C6D1C2078002816
:10AE7000F5D1284611B0F0BD00270121484A0097BE
:10AE800000E00743641C23780846203B98401042AA
:10AE9000F7D120782E2817D1042007436078641C4E
:10AEA0002A280CD10E98641C02C800910E900BE069
:10AEB00000990A22514330394018641C00902078D0
:10AEC000014630390929F3D920780028D1D06428E7
:10AED00008D0692806D075281ED0109A0F9990477F
:10AEE0006D1C5BE00A200E99019001C90E910028AB
:10AEF00002DA40422D2102E0390504D52B216A46B1
:10AF00001172012103E0F90704D02021F7E70BAE0D
:10AF10000B910DE00021FAE70A200E99019001C97A
:10AF20000E91F7E70199FAF7E3F83031761E3170A8
:10AF30000028F7D103A8801B20300190780701D5A5
:10AF4000009801E0012000900199884201DD401A3B
:10AF500000E000200027009006E002A8109AC05DE3
:10AF60000F9990476D1C7F1C0B988742F5DB04E01E
:10AF7000109A30200F9990476D1C0099481E009040
:10AF80000029F5DC05E03078109A761C0F9990477F
:10AF90006D1C0199481E01900029F4DC641C65E7D2
:10AFA00009280100F8B54A002B4B520DD6182B4A40
:10AFB0000C460546142E2BDA002E12DA284BFAF72F
:10AFC000B9F900221346FAF7E5FB40D2002C03DA68
:10AFD0000124E40700253AE02046284337D0214CDD
:10AFE00014E0214F0B46F7403B402B4331D01C4B24
:10AFF000FAF7A0F900221346FAF7CCFB27D2002C6F
:10B0000003DD01200005F0400419BC4300251EE0CB
:10B01000332E1EDC33460027143BFF43DF4038420B
:10B0200017D00F4BFAF730FA00221346FAF7B2FBAB
:10B030000DD2002C0ADD142E0CD03420811B0120EF
:10B0400088404019A84200D2641C0546BD432146F1
:10B050002846F8BD641CF9E701FCFFFF9C750088D9
:10B060003CE4377E0000F03FFFFF0F0070B5044660
:10B070007D20C00060430546284600F001F870BD01
:10B08000002100BF40E000BF00BF00BF00BF00BF05
:10B0900000BF00BF00BF00BF00BF00BF00BF00BFB8
:10B0A00000BF00BF00BF00BF00BF00BF00BF00BFA8
:10B0B00000BF00BF00BF00BF00BF00BF00BF00BF98
:10B0C00000BF00BF00BF00BF00BF00BF00BF00BF88
:10B0D00000BF00BF00BF00BF00BF00BF00BF00BF78
:10B0E00000BF00BF00BF00BF00BF00BF00BF00BF68
:10B0F00000BF00BF00BF00BF00BF00BF00BF00BF58
:10B1000000BF00BF00BF491C8142BCD37047000094
:10B11000F0B585B00446002004900390257860794E
:10B1200040008A49085A02906078401E8849C6B299
:10B130000863042D01D0072D01D1012000E000207B
:10B140000190207882490873E07900280AD10846E6
:10B1500080690121890508437D4988610298C010F2
:10B16000029006E07A488069012189058843784980
:10B170008861207A7649487308468069217A0904F3
:10B1800003221204114008437149886108460021D6
:10B190008269042000F0B5FB6E492E20029A00F06F
:10B1A0009FFB3046FFF788FD6B48405D81004018EB
:10B1B0006A494318052207212B2000F0B7FB684994
:10B1C00001980B1801220B21282000F0AFFB6248E8
:10B1D000405D800063490A580C21282000F091FB53
:10B1E000E079800060494018A1794900425A022163
:10B1F000272000F075FB70005C490A5A04212720C3
:10B2000000F06EFBE079002805D16422062127209A
:10B2100000F066FB1EE0A07804280DD110200090FD
:10B2200010220621272000F05BFB6B46012226211D
:10B23000272000F07BFB0DE0282000902022062133
:10B24000272000F04DFB6B4601222621272000F02D
:10B250006DFB00BF300146494018E1788900425833
:10B260000821272000F04DFBA17A627A08021043E2
:10B27000002803D13F496172090AA172A17A637A59
:10B280000802184302462021272000F029FB3A48F3
:10B290000C210268232000F034FB71003648001DA9
:10B2A000425A0421232000F01BFBA07900280BD078
:10B2B000E0793249431801220021212000F036FBB9
:10B2C00003200490012003902807000F2901F02299
:10B2D0001140084361788904032292041140084315
:10B2E0000499090592001140084303994904012279
:10B2F000520411400843217989051F22920511400B
:10B3000008436179C906C90EC906084307463A468B
:10B3100000211F2000F0F5FAA078617808430004AE
:10B320000B49086108460069E17949030122D2030B
:10B3300011430843064908610846002102690820B4
:10B3400000F0DFFA002005B0F0BD000010BE0008DC
:10B350008C01002004280000B8BD00080200002075
:10B3600020000020C0BD0008E0BD0008ECBD0008C2
:10B37000F0BD000841100000D8BD000822000020E8
:10B3800038B504460D460848808B04432246002108
:10B390002C2000F0A5FA00956B46012206212C20F6
:10B3A00000F0C4FA38BD00008C01002010B5FFF792
:10B3B00071FC10BD70B505460421362000F022F95D
:10B3C0000446002D03D00120C002044304E0012103
:10B3D000C90220468843044622460421362000F054
:10B3E00090FA70BD38B54020009000210E2000F08A
:10B3F00009F90446002211460E2000F082FA6B463D
:10B40000012200210D2000F091FA084A00210F20AE
:10B4100000F077FA00F048FA224600210E2000F0F2
:10B4200070FA00210248017338BD0000F8FF27249C
:10B43000AC010020F0B585B006460420029000273C
:10B44000002001905F494875086300215D48203065
:10B450004171017300205B4988834863886300F071
:10B46000EBF85849086003E000F0E6F85549086039
:10B470005448006854498842F6D10020FFF73CFC4C
:10B4800052480078242804DD504800780446243CC3
:10B490000DE006214D480078F9F740FE0621081A14
:10B4A00045014A480078F9F739FE2C460C4320063E
:10B4B00021040843210208432043039000211E2059
:10B4C000039A00F01EFA02AB01220021242000F0B2
:10B4D0002DFA1E20FFF798FC87B23812394988737D
:10B4E0000420FFF791FC01900198C0B200280FD012
:10B4F000022000906B46012212212D2000F016FA46
:10B500003048808B0121090308432E49888300BFFE
:10B5100000F092F82B4908600620FFF775FC2949D6
:10B5200048600720FFF770FC26498860F806C00EC7
:10B5300008750846007D002801D1102008752149B2
:10B54000087D00F04BFAF007C00F002809D0FFF784
:10B5500042FC1C48808B0121C90208431949888399
:10B560000CE00521362000F035F805461848054066
:10B570002A460521362000F0B3F900BF0120FFF76D
:10B58000BBFB0021042000F03DF80E49886100213A
:10B59000262000F037F8054605208003054380008B
:10B5A00005432A460021262000F0ABF9002226217F
:10B5B000362000F095F900F03FF8024908600020BD
:10B5C00005B0F0BD8C0100203001CADE0100002072
:10B5D000FFFD0000F8B504460D46094FA9B2A0B220
:10B5E0006B46022200F02EF80646002E06D1684671
:10B5F0004078010268460078081887B23846F8BDDE
:10B60000FFFF0000FEB505460E460027FF43B1B21E
:10B61000A8B201AB042200F015F8009000980028B1
:10B6200008D1032404E0380201A9095D4718641E0B
:10B63000002CF8DA3846FEBD10B500210846FFF7A9
:10B64000E1FF10BDFFB581B006460C461746002548
:10B65000002C04D129466D1C684646541AE040204F
:10B660003043C2B229466D1C684642547F2C04DC2C
:10B6700028466D1C69460C540CE0E0B2802108435A
:10B6800029466D1C6A4650546004020E28466D1C03
:10B6900069460A54A8B23A466946049B00F00CFB7E
:10B6A00005B0F0BD70B504460D46164623462A4641
:10B6B00031461120FFF7C6FF70BD10B50446234682
:10B6C000052200211520FFF7BDFF10BD10B5012197
:10B6D0000620FFF797FF10BD10B50446234605224C
:10B6E00000211720FFF7AEFF10BD38B5044600203B
:10B6F000009000F0D9F8FF250135002C01D068003A
:10B7000005432A4600210D2000F0EAF8002C17D04E
:10B710006B46012203210F20FFF794FF6846007853
:10B720000821084000280BD0FFF75CFEFF250135FB
:10B730002A4600210D2000F0D3F80020C04338BD78
:10B740000020FCE710B50446224601210A2000F043
:10B75000D8F810BD70B5054600211A20FFF752FF3A
:10B760000446240D24052803000B0443224600212F
:10B770001A2000F0C6F870BD10B5044622460249F2
:10B780002E2000F0ADF810BD0418000038B50446B6
:10B790006B46012203210420FFF754FF002C16DD25
:10B7A000224600210C2000F09BF869460878102101
:10B7B000084300900F488069090608430D498861D5
:10B7C0006B4601220321042000F0B0F810E0694626
:10B7D000087810218843009006488069090688434C
:10B7E000044988616B4601220321042000F09EF881
:10B7F00038BD00008C01002010B50446224600210F
:10B80000182000F06DF810BDF8B5044600250020A2
:10B81000009000260220204000280AD080200090BE
:10B820006B46012200210D2000F080F801211D4807
:10B830000173E007C00F002826D06946087806216A
:10B84000084300906B46012200210D2000F06EF8A5
:10B8500003210F20FFF7BEFE06468120C0003040C6
:10B86000002801D100251AE0402000906B460122FB
:10B8700000210D2000F05AF80020FFF79BFD002169
:10B88000084801734D1E0AE0694608780221084302
:10B8900000906B46012200210D2000F047F8284659
:10B8A000F8BD0000AC0100201CB501AB0122032152
:10B8B0000F20FFF7C7FE69460879802108406946D6
:10B8C0000979402211404900884208D001200090A7
:10B8D0006B46012203210D2000F028F800BF1CBD9B
:10B8E000F8B505460E4614466846047021124170AC
:10B8F000B1B2A8B26B46022200F018F807463846EB
:10B90000F8BDFEB506460F461446002503E069461D
:10B910004C55240A6D1C042DF9DBB9B2B0B26B464C
:10B92000042200F003F801900198FEBDFFB581B03C
:10B9300006460C4617460025002C07D180203043D0
:10B94000C2B229466D1C6846425419E0C0203043FB
:10B95000C2B228466D1C69460A547F2C03DC284677
:10B960006D1C0C540CE0E0B28021084329466D1C8C
:10B970006A4650546004020E28466D1C69460A54FB
:10B98000A8B23A466946049B00F0E4F905B0F0BD60
:10B9900070B504460E4615462819012189028842D1
:10B9A00002DD0020C04370BDA21E33462946092097
:10B9B000FFF7BCFF0020F6E770B504460D460648C9
:10B9C00000692043A90508430646324600210820A5
:10B9D000FFF797FF002070BD8C01002038B50446AA
:10B9E0006B4601220E212B20FFF72CFE68460078C3
:10B9F000410949010091E106C90E684600780143FA
:10BA000000916B4601220E212B20FFF78FFF38BDDE
:10BA100070B50146002006E00A541E06140A34439D
:10BA20001B0A2246401C0428F6DB70BD13B50C46E9
:10BA300001231A4669460248FCF7ACFD00981CBD7C
:10BA4000101700207CB500210C460D466846FFF714
:10BA500034FE042608E0220E280210432402054684
:10BA60006846805D0443761E002EF4DA204629469F
:10BA70007CBD7CB500210C460D466846FFF72CFEC8
:10BA8000042608E0220E28021043240205466846D8
:10BA9000805D0443761E002EF4DA204629467CBDE4
:10BAA000FBF73AFAFEF736FAFDF7A0F9FDF77EFA52
:10BAB000FDF782F9FDF7C0FAFDF794FAFDF734F9C6
:10BAC0000122D10305200007FBF711FAFEF75EF80B
:10BAD000FCF7F2FFFAF78CF8FAF74EF80721FF208F
:10BAE0004130FFF74DFC2E4800880A2148432D497C
:10BAF00008800122110305200007FBF7F8F9C8228E
:10BB000029492A48FCF7D0FC002801D0FAF7B4F8FC
:10BB100045E02748007800283FD0FEF7FBF90020D9
:10BB200023490870FAF720FB22490870084600787C
:10BB30000F280DDD012211031F48FBF7D8F9FEF78E
:10BB40007BFA0022012109031B48FBF7D0F90CE026
:10BB5000012251031848FBF7CAF9FEF76DFA0022DB
:10BB6000012149031448FBF7C2F9FCF7A7FE0D4871
:10BB70000088002804DD0B480088401E0949088021
:10BB80000E48007800280AD106480088002806D10F
:10BB900001210846FBF756FC01E0FCF78FFEB8E7F1
:10BBA0005C01002070010020F00C00201017002024
:10BBB0004D0100204C0100200004005045000020F1
:10BBC00000B585B01748FBF776FA14216846F9F7F7
:10BBD00002FB154800900320019000200290694666
:10BBE00005200007FBF784F869461048FBF780F84A
:10BBF00069460F48FBF77CF801210846FBF722FC59
:10BC0000FF200130FBF7F0FB0A48006804210843DD
:10BC1000084908608815FBF7F9FBFBF7FFFB05B047
:10BC200000BD000088160020FFFF00000004005047
:10BC3000000800500070004010B5012292021B491C
:10BC40001B48FAF750F8194800881A4988422CD046
:10BC500008461649088004208880FF20F530C880F7
:10BC60000A200881002048811E20C04388810120CD
:10BC7000C88100200884088248828882C88208839C
:10BC800088834320C88602200887782048870120BF
:10BC90008887C88700210548403001844184818419
:10BCA00000200249C88300F03BF810BDB80D002009
:10BCB00000FC0008AA55000070B504460D4600219E
:10BCC000102005263607B06200BF0DE0685C134EF9
:10BCD000F06000BF11488068C007C00F0028F9D08D
:10BCE0000E48C0681870491CA142EFDB00210DE02E
:10BCF00000200A4EF06000BF08488068C007C00FEF
:10BD00000028F9D00548C0685854491C9142EFD327
:10BD1000102005263607B061002070BD00300140BC
:10BD200010B5002472B6012189020848F9F7C0FF56
:10BD30000446002C06D00122920205490348FAF776
:10BD4000A9F8044662B6204610BD000000FC0008B9
:10BD5000B80D002070B504460D46002110200526C0
:10BD60003607B06200BF0CE0685C124EF06000BFA6
:10BD700010488068C007C00F0028F9D00D48C0687F
:10BD8000491CA142F0DB00210CE0585C094EF06038
:10BD900000BF08488068C007C00F0028F9D00548D8
:10BDA000C068491C9142F0D3102005263607B061C7
:10BDB000002070BD003001400000010203040005B6
:10BDC000405C0000A05C0400C06C0800805C0400C3
:10BDD000E03F1E00E07D1E0007A9022570889B88B9
:10BDE0000A001600010006000100020087008D0015
:10BDF0002D001A3152001A339A001A351D011A37D4
:10BE00006B003B31BE003B335E013B3596023B3756
:10BE1000000099599959EB518F421E45142E00800C
:10BE2000EB51F5283333E13A703DE13AC235852BC9
:10BE3000C2353333C235C235AE47E13A5138A3304B
:10BE40005138000000000000000001020304060752
:10BE500008090000000001020304030406080C1096
:10BE60001820300084BE0008000000208C01000073
:10BE7000E8590008C0BE00088C010020AC1A000080
:10BE800086AC000821130704380D091E0805400878
:10BE90002609104008560A131D043B08BE0596D813
:10BEA000BC401008042FC8420115010202141309F6
:10BEB00009120202C9817B8C0ADE01475220000070
:04000005080050C1DE
:00000001FF
